 pcie950_ser

 Timestamp is 4753f239 (Mon Dec 03 12:10:33 2007)

 Preferred load address is 10000000

 Start         Length     Name                   Class
 0001:00000000 0000046cH .rdata                  CODE
 0001:0000046c 00000061H .rdata$debug            CODE
 0001:000004d0 00004f98H .text                   CODE
 0001:00005468 00000028H .idata$2                CODE
 0001:00005490 00000014H .idata$3                CODE
 0001:000054a4 000000c4H .idata$4                CODE
 0001:00005568 000000acH .idata$6                CODE
 0001:00005620 00000107H .edata                  CODE
 0002:00000000 000000c4H .idata$5                DATA
 0002:000000c4 00000004H .CRT$XCA                DATA
 0002:000000c8 00000004H .CRT$XCZ                DATA
 0002:000000cc 00000004H .CRT$XIA                DATA
 0002:000000d0 00000004H .CRT$XIZ                DATA
 0002:000000d4 00000004H .CRT$XPA                DATA
 0002:000000d8 00000004H .CRT$XPZ                DATA
 0002:000000dc 00000004H .CRT$XTA                DATA
 0002:000000e0 00000004H .CRT$XTZ                DATA
 0002:000000e4 00000004H .data                   DATA
 0002:000000e8 00000054H .bss                    DATA

  Address         Publics by Value              Rva+Base     Lib:Object

 0000:00000000       __except_list              00000000     <absolute>
 0001:0000001c       ??_C@_1BI@LAHN@?$AAP?$AAr?$AAi?$AAo?$AAr?$AAi?$AAt?$AAy?$AA2?$AA5?$AA6?$AA?$AA@ 1000101c     mdd.obj
 0001:00000034       ??_C@_1CC@CKAL@?$AAD?$AAe?$AAv?$AAi?$AAc?$AAe?$AAA?$AAr?$AAr?$AAa?$AAy?$AAI?$AAn?$AAd?$AAe?$AAx?$AA?$AA@ 10001034     mdd.obj
 0001:00000224       ??_C@_1CE@GCBE@?$AAF?$AAl?$AAo?$AAw?$AAC?$AAt?$AAr?$AAl?$AAH?$AAi?$AAg?$AAh?$AAL?$AAe?$AAv?$AAe?$AAl?$AA?$AA@ 10001224     ser16950.obj
 0001:00000248       ??_C@_1CC@MJNM@?$AAF?$AAl?$AAo?$AAw?$AAC?$AAt?$AAr?$AAl?$AAL?$AAo?$AAw?$AAL?$AAe?$AAv?$AAe?$AAl?$AA?$AA@ 10001248     ser16950.obj
 0001:0000026c       ??_C@_1BO@HEHB@?$AAR?$AAx?$AAI?$AAn?$AAt?$AAT?$AAr?$AAi?$AAg?$AAL?$AAe?$AAv?$AAe?$AAl?$AA?$AA@ 1000126c     ser16950.obj
 0001:0000028c       ??_C@_1BO@EEEJ@?$AAT?$AAx?$AAI?$AAn?$AAt?$AAT?$AAr?$AAi?$AAg?$AAL?$AAe?$AAv?$AAe?$AAl?$AA?$AA@ 1000128c     ser16950.obj
 0001:000002ac       ??_C@_1CE@MAOK@?$AAB?$AAa?$AAu?$AAd?$AAr?$AAa?$AAt?$AAe?$AAM?$AAa?$AAp?$AAL?$AAi?$AAs?$AAt?$AAT?$AAo?$AA?$AA@ 100012ac     ser16950.obj
 0001:000002d0       ??_C@_1CI@IFEI@?$AAB?$AAa?$AAu?$AAd?$AAr?$AAa?$AAt?$AAe?$AAM?$AAa?$AAp?$AAL?$AAi?$AAs?$AAt?$AAF?$AAr?$AAo?$AAm?$AA?$AA@ 100012d0     ser16950.obj
 0001:000002f8       ??_C@_1CC@JFGI@?$AAC?$AAr?$AAy?$AAs?$AAt?$AAa?$AAl?$AAF?$AAr?$AAe?$AAq?$AAu?$AAe?$AAn?$AAc?$AAy?$AA?$AA@ 100012f8     ser16950.obj
 0001:000003e0       _IoVTbl                    100013e0     oxser.obj
 0001:00000458       ??_C@_1BE@MJOB@?$AAR?$AAe?$AAg?$AAS?$AAt?$AAr?$AAi?$AAd?$AAe?$AA?$AA@ 10001458     oxser.obj
 0001:000004d0       _DoTxData                  100014d0 f   mdd.obj
 0001:00000618       _DoRxData                  10001618 f   mdd.obj
 0001:000006b8       _RxBytesAvail              100016b8 f i mdd.obj
 0001:000006dc       _SerialEventHandler        100016dc f   mdd.obj
 0001:000007b5       _StartDispatchThread       100017b5 f   mdd.obj
 0001:00000860       _StopDispatchThread        10001860 f   mdd.obj
 0001:000008d5       _ApplyDCB                  100018d5 f   mdd.obj
 0001:00000977       _COM_Init                  10001977 f   mdd.obj
 0001:00000b94       _COM_Open                  10001b94 f   mdd.obj
 0001:00000db4       _COM_Close                 10001db4 f   mdd.obj
 0001:00000efb       _ProcessExiting            10001efb f   mdd.obj
 0001:00000fee       _COM_Deinit                10001fee f   mdd.obj
 0001:000010d8       _COM_Read                  100020d8 f   mdd.obj
 0001:00001303       _COM_Write                 10002303 f   mdd.obj
 0001:0000148c       _COM_Seek                  1000248c f   mdd.obj
 0001:00001490       _COM_PowerUp               10002490 f   mdd.obj
 0001:000014a2       _COM_PowerDown             100024a2 f   mdd.obj
 0001:000014bc       _WaitCommEvent             100024bc f   mdd.obj
 0001:000015b9       _EvaluateEventFlag         100025b9 f   mdd.obj
 0001:0000164a       _COM_IOControl             1000264a f   mdd.obj
 0001:00001d59       _OxserGetBaudConfigFromBaudRate 10002d59 f   ser16950.obj
 0001:00001e5c       _ReadPortChar              10002e5c f   ser16950.obj
 0001:00001e67       _ReadRegisterChar          10002e67 f   ser16950.obj
 0001:00001e72       _WritePortChar             10002e72 f   ser16950.obj
 0001:00001e82       _WriteRegisterChar         10002e82 f   ser16950.obj
 0001:00001e92       _ClearPendingInts          10002e92 f   ser16950.obj
 0001:00001f4a       _ReadLSR                   10002f4a f i ser16950.obj
 0001:00001fbe       _ProcessLSR                10002fbe f i ser16950.obj
 0001:00002011       _ReadMSR                   10003011 f i ser16950.obj
 0001:0000208a       _ProcessMSR                1000308a f i ser16950.obj
 0001:000020bd       _InstallSoftwareISR        100030bd f   ser16950.obj
 0001:00002279       _SL_Open                   10003279 f   ser16950.obj
 0001:000024a1       _OUTB_650_REG              100034a1 f i ser16950.obj
 0001:00002554       _OUTB_ICR_REG              10003554 f i ser16950.obj
 0001:000025eb       _SL_Close                  100035eb f   ser16950.obj
 0001:00002696       _SL_Init                   10003696 f   ser16950.obj
 0001:00002781       _SL_PostInit               10003781 f   ser16950.obj
 0001:0000278f       _SL_ClearDTR               1000378f f   ser16950.obj
 0001:00002827       _SL_SetDTR                 10003827 f   ser16950.obj
 0001:000028bf       _SL_ClearRTS               100038bf f   ser16950.obj
 0001:00002957       _SL_SetRTS                 10003957 f   ser16950.obj
 0001:000029ef       _SL_ClearBreak             100039ef f   ser16950.obj
 0001:00002a87       _SL_SetBreak               10003a87 f   ser16950.obj
 0001:00002b1f       _SetBaudRate               10003b1f f   ser16950.obj
 0001:00002b7f       _WRITE_DIVISOR_REG         10003b7f f i ser16950.obj
 0001:00002c43       _SL_SetBaudRate            10003c43 f   ser16950.obj
 0001:00002cd0       _SL_SetByteSize            10003cd0 f   ser16950.obj
 0001:00002da6       _SL_SetParity              10003da6 f   ser16950.obj
 0001:00002e85       _SL_SetStopBits            10003e85 f   ser16950.obj
 0001:00002f4c       _SL_GetRxBufferSize        10003f4c f   ser16950.obj
 0001:00002f52       _SL_GetInterruptType       10003f52 f   ser16950.obj
 0001:0000306b       _ReadASR                   1000406b f i ser16950.obj
 0001:00003137       _SL_RxIntr                 10004137 f   ser16950.obj
 0001:0000342f       _BytesInFifo               1000442f f i ser16950.obj
 0001:000034f6       _SL_TxIntrEx               100044f6 f   ser16950.obj
 0001:00003763       _SL_LineIntr               10004763 f   ser16950.obj
 0001:000037e9       _SL_OtherIntr              100047e9 f   ser16950.obj
 0001:000038e5       _SL_ModemIntr              100048e5 f   ser16950.obj
 0001:000038f0       _SL_GetStatus              100048f0 f   ser16950.obj
 0001:00003a0d       _INB_650_REG               10004a0d f i ser16950.obj
 0001:00003ac1       _SL_Reset                  10004ac1 f   ser16950.obj
 0001:00003b86       _SL_GetModemStatus         10004b86 f   ser16950.obj
 0001:00003bbb       _SL_PurgeComm              10004bbb f   ser16950.obj
 0001:00003cbf       _SL_XmitComChar            10004cbf f   ser16950.obj
 0001:00003e04       _SL_PowerOff               10004e04 f   ser16950.obj
 0001:00003fe3       _SL_PowerOn                10004fe3 f   ser16950.obj
 0001:000041dd       _SL_SetDCB                 100051dd f   ser16950.obj
 0001:000043fe       _SL_SetCommTimeouts        100053fe f   ser16950.obj
 0001:00004418       _SetFifoCtrlLevels         10005418 f   ser16950.obj
 0001:00004544       _SetInternalLoopback       10005544 f   ser16950.obj
 0001:00004571       _SaveBaudrateMap           10005571 f   ser16950.obj
 0001:00004708       _RegSetDeviceValue         10005708 f   ser16950.obj
 0001:0000474f       _SL_Ioctl                  1000574f f   ser16950.obj
 0001:00004947       _SL_EnableXmit             10005947 f   ser16950.obj
 0001:0000497c       _SL_DisableXmit            1000597c f   ser16950.obj
 0001:000049b1       _GetRegMultiDword          100059b1 f   oxser.obj
 0001:00004a29       _Ser_GetRegistryData       10005a29 f   oxser.obj
 0001:0000511f       _Ser_Ioctl                 1000611f f   oxser.obj
 0001:0000521b       _GetSerialObject           1000621b f   oxser.obj
 0001:0000523e       _LeaveCriticalSection      1000623e f   coredll:COREDLL.dll
 0001:00005244       _EventModify               10006244 f   coredll:COREDLL.dll
 0001:0000524a       _SetProcPermissions        1000624a f   coredll:COREDLL.dll
 0001:00005250       _EnterCriticalSection      10006250 f   coredll:COREDLL.dll
 0001:00005256       _ExitThread                10006256 f   coredll:COREDLL.dll
 0001:0000525c       _CreateThread              1000625c f   coredll:COREDLL.dll
 0001:00005262       _InterruptDone             10006262 f   coredll:COREDLL.dll
 0001:00005268       _InterruptInitialize       10006268 f   coredll:COREDLL.dll
 0001:0000526e       _InterruptDisable          1000626e f   coredll:COREDLL.dll
 0001:00005274       _LocalFree                 10006274 f   coredll:COREDLL.dll
 0001:0000527a       _OpenDeviceKey             1000627a f   coredll:COREDLL.dll
 0001:00005280       _InitializeCriticalSection 10006280 f   coredll:COREDLL.dll
 0001:00005286       _LocalAlloc                10006286 f   coredll:COREDLL.dll
 0001:0000528c       _DeleteCriticalSection     1000628c f   coredll:COREDLL.dll
 0001:00005292       _GetCurrentPermissions     10006292 f   coredll:COREDLL.dll
 0001:00005298       __except_handler3          10006298 f   coredll:COREDLL.dll
 0001:0000529e       _FreePhysMem               1000629e f   coredll:COREDLL.dll
 0001:000052a4       _LoadIntChainHandler       100062a4 f   coredll:COREDLL.dll
 0001:000052aa       _KernelLibIoControl        100062aa f   coredll:COREDLL.dll
 0001:000052b0       _wcslen                    100062b0 f   coredll:COREDLL.dll
 0001:000052b6       __ultow                    100062b6 f   coredll:COREDLL.dll
 0001:000052bc       _wcstoul                   100062bc f   coredll:COREDLL.dll
 0001:000052c2       _DDKReg_GetWindowInfo      100062c2 f   coredll:COREDLL.dll
 0001:000052c8       _wcscpy                    100062c8 f   coredll:COREDLL.dll
 0001:000052ce       _DDKReg_GetIsrInfo         100062ce f   coredll:COREDLL.dll
 0001:000052d4       _VirtualFree               100062d4 f   coredll:COREDLL.dll
 0001:000052da       _READ_PORT_UCHAR           100062da f   ceddk:CEDDK.dll
 0001:000052e0       _READ_REGISTER_UCHAR       100062e0 f   ceddk:CEDDK.dll
 0001:000052e6       _WRITE_PORT_UCHAR          100062e6 f   ceddk:CEDDK.dll
 0001:000052ec       _WRITE_REGISTER_UCHAR      100062ec f   ceddk:CEDDK.dll
 0001:000052f2       _TransBusAddrToStatic      100062f2 f   ceddk:CEDDK.dll
 0001:000052f8       _TransBusAddrToVirtual     100062f8 f   ceddk:CEDDK.dll
 0001:000052fe       _MmUnmapIoSpace            100062fe f   ceddk:CEDDK.dll
 0001:00005304       __DllMainCRTStartup        10006304 f   corelibc:pegdmain.obj
 0001:00005374       __abnormal_termination     10006374 f   corelibc:_exclst_.obj
 0001:00005379       __cinit                    10006379 f   corelibc:crt0dat.obj
 0001:0000543d       __cexit                    1000643d f   corelibc:crt0dat.obj
 0001:0000544c       _DllMain                   1000644c f   corelibc:dllmain.obj
 0001:00005462       ___abnormal_termination    10006462 f   coredll:COREDLL.dll
 0001:00005468       __IMPORT_DESCRIPTOR_COREDLL 10006468     coredll:COREDLL.dll
 0001:0000547c       __IMPORT_DESCRIPTOR_CEDDK  1000647c     ceddk:CEDDK.dll
 0001:00005490       __NULL_IMPORT_DESCRIPTOR   10006490     coredll:COREDLL.dll
 0002:00000000       __imp__TransBusAddrToVirtual 10007000     ceddk:CEDDK.dll
 0002:00000004       __imp__TransBusAddrToStatic 10007004     ceddk:CEDDK.dll
 0002:00000008       __imp__WRITE_REGISTER_UCHAR 10007008     ceddk:CEDDK.dll
 0002:0000000c       __imp__WRITE_PORT_UCHAR    1000700c     ceddk:CEDDK.dll
 0002:00000010       __imp__READ_REGISTER_UCHAR 10007010     ceddk:CEDDK.dll
 0002:00000014       __imp__READ_PORT_UCHAR     10007014     ceddk:CEDDK.dll
 0002:00000018       __imp__MmUnmapIoSpace      10007018     ceddk:CEDDK.dll
 0002:0000001c       \177CEDDK_NULL_THUNK_DATA  1000701c     ceddk:CEDDK.dll
 0002:00000020       __imp__InterruptInitialize 10007020     coredll:COREDLL.dll
 0002:00000024       __imp__WaitForSingleObject 10007024     coredll:COREDLL.dll
 0002:00000028       __imp__Sleep               10007028     coredll:COREDLL.dll
 0002:0000002c       __imp__InterruptDisable    1000702c     coredll:COREDLL.dll
 0002:00000030       __imp__CloseHandle         10007030     coredll:COREDLL.dll
 0002:00000034       __imp__CeSetThreadPriority 10007034     coredll:COREDLL.dll
 0002:00000038       __imp__CeGetThreadPriority 10007038     coredll:COREDLL.dll
 0002:0000003c       __imp__LocalFree           1000703c     coredll:COREDLL.dll
 0002:00000040       __imp__RegCloseKey         10007040     coredll:COREDLL.dll
 0002:00000044       __imp__RegQueryValueExW    10007044     coredll:COREDLL.dll
 0002:00000048       __imp__OpenDeviceKey       10007048     coredll:COREDLL.dll
 0002:0000004c       __imp__CreateEventW        1000704c     coredll:COREDLL.dll
 0002:00000050       __imp__InitializeCriticalSection 10007050     coredll:COREDLL.dll
 0002:00000054       __imp__LocalAlloc          10007054     coredll:COREDLL.dll
 0002:00000058       __imp__DeleteCriticalSection 10007058     coredll:COREDLL.dll
 0002:0000005c       __imp__SetLastError        1000705c     coredll:COREDLL.dll
 0002:00000060       __imp__InterruptDone       10007060     coredll:COREDLL.dll
 0002:00000064       __imp__GetTickCount        10007064     coredll:COREDLL.dll
 0002:00000068       __imp__GetCurrentPermissions 10007068     coredll:COREDLL.dll
 0002:0000006c       __imp___except_handler3    1000706c     coredll:COREDLL.dll
 0002:00000070       __imp__FreePhysMem         10007070     coredll:COREDLL.dll
 0002:00000074       __imp__LoadIntChainHandler 10007074     coredll:COREDLL.dll
 0002:00000078       __imp__KernelLibIoControl  10007078     coredll:COREDLL.dll
 0002:0000007c       __imp__wcslen              1000707c     coredll:COREDLL.dll
 0002:00000080       __imp___ultow              10007080     coredll:COREDLL.dll
 0002:00000084       __imp__RegSetValueExW      10007084     coredll:COREDLL.dll
 0002:00000088       __imp__wcstoul             10007088     coredll:COREDLL.dll
 0002:0000008c       __imp__DDKReg_GetWindowInfo 1000708c     coredll:COREDLL.dll
 0002:00000090       __imp__wcscpy              10007090     coredll:COREDLL.dll
 0002:00000094       __imp__DDKReg_GetIsrInfo   10007094     coredll:COREDLL.dll
 0002:00000098       __imp__VirtualFree         10007098     coredll:COREDLL.dll
 0002:0000009c       __imp__CreateThread        1000709c     coredll:COREDLL.dll
 0002:000000a0       __imp__ExitThread          100070a0     coredll:COREDLL.dll
 0002:000000a4       __imp__EnterCriticalSection 100070a4     coredll:COREDLL.dll
 0002:000000a8       __imp__SetProcPermissions  100070a8     coredll:COREDLL.dll
 0002:000000ac       __imp__EventModify         100070ac     coredll:COREDLL.dll
 0002:000000b0       __imp__LeaveCriticalSection 100070b0     coredll:COREDLL.dll
 0002:000000b4       __imp__SetThreadPriority   100070b4     coredll:COREDLL.dll
 0002:000000b8       __imp__DisableThreadLibraryCalls 100070b8     coredll:COREDLL.dll
 0002:000000bc       __imp____abnormal_termination 100070bc     coredll:COREDLL.dll
 0002:000000c0       \177COREDLL_NULL_THUNK_DATA 100070c0     coredll:COREDLL.dll
 0002:000000c4       ___xc_a                    100070c4     corelibc:crt0init.obj
 0002:000000c8       ___xc_z                    100070c8     corelibc:crt0init.obj
 0002:000000cc       ___xi_a                    100070cc     corelibc:crt0init.obj
 0002:000000d0       ___xi_z                    100070d0     corelibc:crt0init.obj
 0002:000000d4       ___xp_a                    100070d4     corelibc:crt0init.obj
 0002:000000d8       ___xp_z                    100070d8     corelibc:crt0init.obj
 0002:000000dc       ___xt_a                    100070dc     corelibc:crt0init.obj
 0002:000000e0       ___xt_z                    100070e0     corelibc:crt0init.obj
 0002:0000012c       __exitflag                 1000712c     <common>
 0002:00000130       ___onexitend               10007130     <common>
 0002:00000134       ___onexitbegin             10007134     <common>
 0002:00000138       __pRawDllMain              10007138     <common>

 entry point at        0001:00005304

 Static symbols

 0001:00000814       _SerialDispatchThread      10001814 f   mdd.obj
 0001:00004d9a       _SerInit                   10005d9a f   oxser.obj
 0001:00004ef8       _Ser_InternalMapRegisterAddresses 10005ef8 f   oxser.obj
 0001:00004f68       _SerSetOutputMode          10005f68 f   oxser.obj
 0001:00004f69       _SerClose                  10005f69 f   oxser.obj
 0001:00004fd9       _SerDeinit                 10005fd9 f   oxser.obj
 0001:00005044       _SerGetCommProperties      10006044 f   oxser.obj
 0001:0000505c       _SerPowerOff               1000605c f   oxser.obj
 0001:00005079       _SerPowerOn                10006079 f   oxser.obj
 0001:000050a1       _SerEnableIR               100060a1 f   oxser.obj
 0001:000050c0       _SerDisableIR              100060c0 f   oxser.obj
 0001:000050dc       _SerOpen                   100060dc f   oxser.obj
 0001:0000539b       __initterm                 1000639b f   corelibc:crt0dat.obj
 0001:000053b5       _doexit                    100063b5 f   corelibc:crt0dat.obj
